:1000000015C039C038C0F3C236C035C034C033C0A3
:1000100032C031C030C02FC02EC02DC02CC02BC06C
:100020002AC029C028C09A00F102670411241FBE0B
:10003000CFE5D4E0DEBFCDBF10E0A0E6B0E0ECE756
:10004000F1E102C005900D92AA39B107D9F711E08C
:10005000AAE9B0E001C01D92AA37B107E1F710E0AC
:10006000CCE2D0E003C02297FE0183D8C632D1078C
:10007000D1F751D182C8C4CFE1E1F1E0A8E1B1E00C
:100080008C912081820F912D911D9695879580836B
:100090003197119781E0EA30F80791F708950F93AF
:1000A0001F93019709F043C06F5F7F4F09F03FC076
:1000B00040E063E48AE990E0D0D620E044E064E4E4
:1000C00083EB90E0FCD10CEB12E024EB35E040E058
:1000D00063EB70E08BEB90E0E3D420E042E063E47C
:1000E0008BEC90E0A2D120E043E063E483ED90E06C
:1000F0009CD120E042E064E48BED90E0E0D120E090
:1001000043E064E483EE90E0DAD10CE211E02CED00
:1001100035E041E06BED70E08BEE90E0C1D42CED6A
:1001200035E040E063EE70E08BEF90E0B9D41F91D2
:100130000F9108956FEF7FEF81E090E0B0DF0895B9
:1001400060E070E08BEE90E058D460E070E08BEF00
:1001500090E053D410921E01E1E1F1E0108231975A
:1001600081E0EA30F807D1F70895EF92FF920F93FC
:100170001F936091ED007091EE000091FD001091D1
:10018000FE00FF24EE2421E030E0F901E55FFE4FA0
:100190009081EE2DF0E0E55FFE4F8081981708F426
:1001A000E22EEF2DF0E0E55FFE4F8081891708F425
:1001B000F22E2F5F3F4F2730310539F7EF2DF0E05A
:1001C000E55FFE4F80818F3698F080911D01882376
:1001D00059F4EF1428F460EE7FEF0FE110E004C053
:1001E0006FE170E000EE1FEF81E080931D0115C00C
:1001F0000FE110E02FEF30E04EE650E060E070E0FD
:1002000090E0E0D4BC01EF1418F40FEF10E003C04D
:100210008C016FEF70E010921D018BEE90E0EDD33A
:10022000B8018BEF90E0E9D31F910F91FF90EF9011
:100230000895EF92FF920F931F937B018C018091A1
:10024000190190911A01A0911B01B0911C01A80104
:100250009701281B390B4A0B5B0B2F3131054105E8
:10026000510508F446C08AE990E0DBD5882309F4FB
:1002700040C060E08AE990E010D540E850E060E0DE
:1002800070E0E3D420916E0030916F00F901EE5ED2
:10029000FE4F90E8981B908380911E01873018F4E0
:1002A0008F5F80931E01E0921901F0921A01009372
:1002B0001B0110931C012115310519F481E090E018
:1002C00005C02630310539F48FEF9FEF9093710010
:1002D00080937000D1DE80916E0090916F0020912C
:1002E000700030917100820F931F90936F00809384
:1002F0006E00E0916E00F0916F00EE0FFF1FE05A6C
:10030000FF4F608171818BEB90E077D31F910F914C
:10031000FF90EF900895CF92DF92EF92FF920F93AC
:100320001F93CF93DF93F9D068EE73E097D108DF86
:100330004BEEC42E40E0D42ECBEFD0E0EED0F4D084
:100340007B018C018091D200882371F1E091CC0077
:10035000F091CD00208130E08091CB0090E0282307
:100360003923232B09F160EC7FEFC60146D360EC03
:100370007FEFCE0142D3D1D028EE33E0B801A70100
:10038000DFD0882381F36FEF70E0C60136D361E0E0
:100390007FEFCE0132D3C1D02CED35E0B801A701FB
:1003A000CFD0882381F331C08091DA00882371F1A6
:1003B000E091D400F091D500208130E08091D3000D
:1003C00090E028233923232B09F160EC7FEFC6014D
:1003D00014D360EC7FEFCE0110D39FD028EE33E032
:1003E000B801A701ADD0882381F361E07FEFC6019A
:1003F00004D36FEF70E0CE0100D38FD02CED35E049
:10040000B801A7019DD0882381F39ADEC801B70106
:1004100010DF80911E01873008F0A7DE7ED0A80192
:10042000970164E170E0B2D089CF1F93CF93DF933F
:10043000EC01122F36D58F81882379F0CE01AFD50C
:10044000EB81FC819881112321F08081892B8083AD
:1004500004C08081909598239083DF91CF911F9164
:1004600008951F93CF93DF93EC01122F1AD58F813C
:10047000882379F0CE0193D5EB81FC8198811123FB
:1004800021F08081892B808304C0808190959823FE
:100490009083DF91CF911F910895FC01878188237C
:1004A00069F0A381B4819081662321F08C91892B1E
:1004B0008C9308958C91909598239C9308951F9305
:1004C000CF93DF93EC01122FECD48F81882329F096
:1004D000CE0176D5612FCE01E0DFDF91CF911F9164
:1004E00008951F93CF93DF93EC01122FDAD48F81FD
:1004F000882329F0CE0164D5612FCE01CEDFDF91B4
:10050000CF911F91089514BC8CE085BD8DE783BD0C
:1005100089B7806889BF789408958FE191E0089544
:10052000F2DF0895F0DF08952FB7F894609120016D
:100530007091210180912201909123012FBF089594
:10054000EF92FF920F931F937A018B016FB7F8948C
:100550008091200190912101A0912201B09123016D
:100560006FBF60E070E08E199F09A00BB10B40E0F7
:1005700050E0281739074A075B0710F461E070E084
:10058000CB011F910F91FF90EF900895EF92FF9292
:100590000F931F9379018A01AB0160E070E02FB7E0
:1005A000F8948091200190912101A0912201B091B5
:1005B00023012FBF8E199F09A00BB10B48175907B4
:1005C0006A077B0760F71F910F91FF90EF900895E6
:1005D000019731F46F5F7F4F19F48FE191E0A2DF53
:1005E00008956FEF7FEF81E090E0F2DF08951F92B2
:1005F0000F920FB60F9211242F933F934F935F9357
:100600006F937F938F939F93AF93BF93EF93FF93DA
:100610008091200190912101A0912201B0912301AC
:100620000196A11DB11D8093200190932101A093FB
:100630002201B09323011FD050D1FF91EF91BF91C0
:10064000AF919F918F917F916F915F914F913F916A
:100650002F910F900FBE0F901F901895EFB7F89441
:1006600020912001309121014091220150912301DC
:10067000EFBF8CDF089584E291E00895DC012FB78D
:10068000F89480E090E0FC01EE0FFF1FEE0FFF1FDB
:10069000E80FF91FEA0FFB1F1382128211821082EA
:1006A000848301968031910571F7A05BBF4F1D9245
:1006B0001D92FD0110821182128213822FBF0895B4
:1006C000DC012FB7F89480E090E0FC01EE0FFF1FF3
:1006D000EE0FFF1FE80FF91FEA0FFB1F13821282B4
:1006E00011821082848301968031910571F7A05B9D
:1006F000BF4F1D921D92FD01108211821282138242
:100700002FBF0895EF92FF920F931F93CF93DF9324
:10071000EC018B01BA01FFB6F894C05BDF4F588142
:10072000C055D04020E0852F90E0FC01EE0FFF1F68
:10073000EE0FFF1FE80FF91FEC0FFD1F8281938161
:10074000892B39F02F5F203109F4B0C051505F7010
:10075000EACF503108F0AAC0DE01AF5ABF4F8C91EA
:1007600090E0FC01EE0FFF1FEE0FFF1FE80FF91FD7
:10077000EC0FFD1F82819381892B09F48FC08C912E
:1007800090E0FC01EE0FFF1FEE0FFF1FE80FF91FB7
:10079000EC0FFD1F808191816817790708F47EC0F6
:1007A000EC9022C08D919C91119768177907E0F029
:1007B000FD01848190E08217930711F4E42E14C0A8
:1007C000FD018481E42E482F242F30E0D901AA0FA7
:1007D000BB1FAA0FBB1FA20FB31FAC0FBD1FFD0194
:1007E00082819381892BF1F6852F90E0DC01AA0F9D
:1007F000BB1FAA0FBB1FA80FB91FAC0FBD1FFD0168
:100800001383028311967C936E935483FFEFEF164C
:1008100021F12E2D30E0F901EE0FFF1FEE0FFF1F2B
:10082000E20FF31FEC0FFD1F848190E08217930706
:1008300021F08481FD01848305C0CF5ADF4F5883A6
:10084000C155D040F901EE0FFF1FEE0FFF1FE20F61
:10085000F31FEC0FFD1F548329C09E01205B3F4F07
:10086000F901808190E0FC01EE0FFF1FEE0FFF1FEA
:10087000E80FF91FEC0FFD1F82819381892B29F06E
:10088000F9018081FD01848305C0CF5ADF4F588371
:10089000C155D040C05BDF4F588308C0C05BDF4FFD
:1008A0004881C055D040EE24EA948ECFFFBEDF9140
:1008B000CF911F910F91FF90EF900895019731F420
:1008C0006F5F7F4F19F484E291E0FADE08956FEFD5
:1008D0007FEF81E090E0F2DF08958F929F92AF92D8
:1008E000BF92CF92DF92EF92FF920F931F93CF931D
:1008F000DF935C0112DE18DE9B01AC01F501EE5ABC
:10090000FF4F80819181A281B38179018A01E81A28
:10091000F90A0A0B1B0B09F44BC080819181A2815B
:10092000B381281739074A075B0728F40894E108C0
:10093000F108010911092083318342835383F501B2
:10094000E05BFF4FC0804F0124C0DC80888199812B
:10095000A0E0B0E0E816F9060A071B0788F0EA8174
:10096000FB811B821A8219821882CC82D401DC920C
:10097000A081B1812D913C91CF01F901099506C06B
:10098000888199818E199F0999838883CD1481F07C
:10099000CD2C8C2D90E0EC01CC0FDD1FCC0FDD1F9A
:1009A000C80FD91FCA0DDB1D8A819B81892B69F66F
:1009B000DF91CF911F910F91FF90EF90DF90CF903B
:1009C000BF90AF909F908F900895FC0187818823FE
:1009D00069F0A381B4819081662321F08C91892BE9
:1009E0008C9308958C91909598239C93089561E041
:1009F00054DD089560E051DD0895CF92DF92EF92CB
:100A0000FF920F931F93CF93DF93EC0102D36C01FE
:100A10008C818823D1F1ED80FE800F8118857DDDEA
:100A200024E130E0B801A7018BDD882371F18B85CB
:100A3000882321F0D094C194D108D3942C853D858E
:100A40008E859F858C01020F131F281B390B4FEFDA
:100A500050E061E07FEFC601B5D08C01FFB6F8949D
:100A600089859A85C4DFC80164E170E01CD3CB019D
:100A700068E070E07ED089859A85BCDFFFBE4DDDE1
:100A800053DD6D837E838F8398878A819B81DF917D
:100A9000CF911F910F91FF90EF90DF90CF9008952D
:100AA000AF92BF92DF92EF92FF920F931F93CF937B
:100AB000DF93EC015B01D42E790192D286E790E0BE
:100AC00099838883DB86FD86EC861F870E87F50178
:100AD0008781882369F0BA86A986C5018BDF1DDD71
:100AE00023DD6D837E838F839887CE018ED202C0F3
:100AF0001A861986DF91CF911F910F91FF90EF9089
:100B0000DF90BF90AF900895AF92BF92DF92EF92C7
:100B1000FF920F931F93CF93DF93EC015B01D42ED1
:100B200079015ED286E790E099838883DB86FD8633
:100B3000EC861F870E87F5018781882369F0BA86C6
:100B4000A986C50157DFE9DCEFDC6D837E838F83E7
:100B50009887CE015AD202C01A861986DF91CF91AA
:100B60001F910F91FF90EF90DF90BF90AF9008958D
:100B70000895CF93DF93CDB7DEB722970FB6F894E1
:100B8000DEBF0FBECDBF9A83898389819A819C0184
:100B9000629FC001639F900D729F900D112403C04E
:100BA00089819A8101979A83898389819A81892B86
:100BB000B9F722960FB6F894DEBF0FBECDBFDF9116
:100BC000CF9108954F925F926F927F928F929F92F2
:100BD000AF92BF92CF92DF92EF92FF920F931F934B
:100BE0002B015A0139017801E21AF30A0027F7FCB8
:100BF0000095102F9C01261B370B442737FD40958D
:100C0000542FC801B70130D2A418B508CC24B7FCC2
:100C1000C094DC2CA60195017BD2882477FC8094BB
:100C2000982C620E731E841E951EC3011F910F9196
:100C3000FF90EF90DF90CF90BF90AF909F908F90FC
:100C40007F906F905F904F900895681779070CF42C
:100C5000BC01461757070CF4BA01CB010895CF9396
:100C6000DF93DC01EC018F81882319F420E030E070
:100C70000EC0ED01E981FA8120818C9130E090E095
:100C8000282339232115310511F021E030E081E0DE
:100C9000822790E0DF91CF9108951F93CF93DF9348
:100CA000EC01162FE881F9810190F081E02D099582
:100CB00024E630E0829FB001839F700D929F700DFB
:100CC000112480E090E022E831E040E050E0FED1E5
:100CD000C9011123D1F1688D67FF0DC0188EFE0187
:100CE00020E030E0918B808B2F5F3F4F3296283091
:100CF000310559F1F7CFE62FFF27E7FDF095EE0F0D
:100D0000FF1FEC0FFD1F318B208B6F5F6770688FAB
:100D1000FE0120E030E040E050E060E070E08089DB
:100D20009189A0E0B0E0280F391F4A1F5B1F6F5F59
:100D30007F4F32966830710591F783E0569547955D
:100D4000379527958A95D1F7C901DF91CF911F91EA
:100D50000895FF920F931F93CF93DF93EC01898542
:100D6000882309F456C0E881F9810480F581E02DDB
:100D7000CE010995882309F44CC0EF81F885808164
:100D80009A81892B8083ED81FE8190818A81809573
:100D900089238083FFB6F894ED81FE8180819A815A
:100DA000892B808368E070E081E090E0E2DEED81F5
:100DB000FE8190818A81809589238083EF81F885E7
:100DC00090818A818095892380838E010E5F1F4FD9
:100DD000C80145DF8823E1F740E050E002C04F5FE3
:100DE0005F4FEB81FC8120818A8130E090E02823F5
:100DF0003923232BA1F7FFBE23E0569547952A956B
:100E0000E1F75F874E8789DB8FDB6A877B878C877B
:100E10009D878E859F85DF91CF911F910F91FF90C8
:100E20000895EF92FF920F931F93FC01E284F384E5
:100E300004851585E114F1040105110511F481E023
:100E400006C06BDB22E330E0B801A70179DB90E05C
:100E50001F910F91FF90EF9008950F931F938C01B6
:100E6000F5D080E890E0F8019183808312861386A4
:100E7000148615868FEF808F1F910F9108950F9321
:100E80001F938C01E3D080E890E0F8019183808388
:100E900012861386148615868FEF808F1F910F910F
:100EA0000895FC0181E090E002C0880F991F4A95E7
:100EB000E2F7808381E08783643419F165342CF490
:100EC000623449F0633451F511C0633679F0643609
:100ED000C1F0623619F587E390E09683858386E357
:100EE00090E09283818388E390E015C084E390E0F2
:100EF0009683858383E390E09283818385E390E00A
:100F00000AC081E390E09683858380E390E092833A
:100F1000818382E390E09483838308951782089508
:100F2000FC0181E090E002C0880F991F4A95E2F72A
:100F3000808381E08783643419F165342CF4623452
:100F400049F0633451F511C0633679F06436C1F06D
:100F5000623619F587E390E09683858386E390E017
:100F60009283818388E390E015C084E390E09683C8
:100F7000858383E390E09283818385E390E00AC0D8
:100F800081E390E09683858380E390E09283818380
:100F900082E390E094838383089517820895CF932A
:100FA000DF93DC01EC018F81882339F0ED81FE8134
:100FB00090818C91809589238083DF91CF910895D2
:100FC000CF93DF93DC01EC018F81882331F0ED8139
:100FD000FE8180819C91892B8083DF91CF91089540
:100FE000FC018AE890E0918380831382128214824C
:100FF0000895FC018AE890E0918380831382128235
:1010000014820895FC011482089521E0FC012483D8
:1010100008950F931F938C01CB014FEF50E061E0D7
:101020007FEF13DEF801938382831F910F91089560
:101030000F931F938C0120E0029613DA84E990E06D
:10104000F801918380831F910F9108950F931F934F
:101050008C0120E0029605DA84E990E0F8019183A2
:1010600080831F910F910895629FD001739FF001BB
:10107000829FE00DF11D649FE00DF11D929FF00D28
:10108000839FF00D749FF00D659FF00D9927729F5F
:10109000B00DE11DF91F639FB00DE11DF91FBD01EA
:1010A000CF011124089597FB092E07260AD077FD5A
:1010B00004D049D006D000201AF4709561957F4F76
:1010C0000895F6F7909581959F4F0895A1E21A2E05
:1010D000AA1BBB1BFD010DC0AA1FBB1FEE1FFF1FDC
:1010E000A217B307E407F50720F0A21BB30BE40B2C
:1010F000F50B661F771F881F991F1A9469F7609573
:101100007095809590959B01AC01BD01CF0108952C
:1011100097FB092E05260ED057FD04D0D7DF0AD045
:10112000001C38F450954095309521953F4F4F4F16
:101130005F4F0895F6F790958095709561957F4F74
:101140008F4F9F4F0895AA1BBB1B51E107C0AA1FD9
:10115000BB1FA617B70710F0A61BB70B881F991F58
:101160005A95A9F780959095BC01CD010895EE0F91
:0C117000FF1F0590F491E02D0994FFCFC3
:10117C0001FF56FFABFF00005500AA00FF00040062
:10118C00010000000000FD0405080208000000003A
:10119C00A9064D06110700000000B8050508020855
:0A11AC0000000000B805B805B80502
:00000001FF
